:100000000C9446030C9465030C9465030C946503EF
:100010000C9465030C9465030C9465030C946503C0
:100020000C9465030C9402040C9465030C94650312
:100030000C9465030C9465030C9465030C946503A0
:100040000C9465030C9465030C9465030C94650390
:100050000C9439040C9465040C9465030C946503AA
:100060000C9465030C9465030C9465030C94650370
:100070000C9465030C9465030C9465030C94650360
:100080000C9465030C9465030C9465030000000058
:100090000000003E4551453E003E6B6F6B3E001C2C
:1000A0003E7C3E1C00183C7E3C180030367F3630CB
:1000B00000185C7E5C1800000000000000000000DA
:1000C0000000000000000000000000000000003000
:1000D000484A360E00062979290600000000000073
:1000E00000607E0A353F002A1C361C2A00007F3E35
:1000F0001C0800081C3E7F000014367F36140000E8
:100100005F005F000006097F017F00224D555922E4
:100110000060606060000014B6FFB6140004067F43
:1001200006040010307F30100008083E1C0800084C
:100130001C3E080800784040404000083E083E0849
:1001400000303C3F3C3000030F3F0F030000000035
:1001500000000000065F06000007030007030024FC
:100160007E247E2400242B6A12000063130864633B
:1001700000364956205000000703000000003E41B1
:1001800000000000413E000000083E1C3E08000840
:10019000083E08080000E0600000000808080808A1
:1001A000000060600000002010080402003E514979
:1001B000453E0000427F400000625149494600220E
:1001C00049494936001814127F10002F4949493116
:1001D000003C4A494930000171090503003649498C
:1001E000493600064949291E00006C6C00000000D9
:1001F000EC6C000000081422410000242424242474
:10020000000041221408000201590906003E415D28
:10021000551E007E1111117E007F49494936003E6E
:1002200041414122007F4141413E007F49494941CE
:10023000007F09090901003E4149497A007F080809
:10024000087F0000417F410000304040403F007F78
:1002500008142241007F40404040007F0204027F9A
:10026000007F0204087F003E4141413E007F0909B2
:100270000906003E4151215E007F090919660026EA
:10028000494949320001017F0101003F4040403FA0
:10029000001F2040201F003F403C403F00631408E7
:1002A0001463000708700807007149454300000007
:1002B0007F414100000204081020000041417F00FE
:1002C0000004020102048080808080800000030717
:1002D0000000002054545478007F444444380038CF
:1002E0004444442800384444447F0038545454085B
:1002F00000087E0909000018A4A4A47C007F04045F
:1003000078000000007D4000004080847D00007F78
:10031000102844000000007F4000007C041804788E
:10032000007C0404780000384444443800FC444411
:1003300044380038444444FC00447844040800082D
:100340005454542000043E442400003C40207C00CF
:10035000001C2040201C003C6030603C006C1010F1
:100360006C00009CA0603C00006454544C000008E9
:100370003E414100000000770000000041413E087E
:10038000000201020100003C2623263C001EA1E1E0
:100390002112003D40207D000038545455090020B2
:1003A00055555578002055545578002055555478AA
:1003B000002057555778001CA2E2221400385555EA
:1003C0005508003855545508003855555408000054
:1003D000017C41000000017D41000000017C4000E3
:1003E00000702924297000782F252F78007C545420
:1003F00055450034547C5458007E097F49490038E3
:100400004545390000384544390000394544380035
:10041000003C41217D00003D41207C00009CA1600A
:100420003D00003D42423D00003C41403D008070A7
:100430006858380400483E494962007E615D433F88
:100440000022140814220040887E0902002054551E
:1004500055780000007D4100003844453900003CDB
:1004600040217D00007A090A7100007A112279008A
:1004700000085555555E004E51514E000030484D14
:1004800040203E415D4B553E04040404041C00170B
:10049000084C6A50001708342A780000307D30007C
:1004A0000008140008140014080014084411441132
:1004B0004411AA55AA55AA55BBEEBBEEBBEE0000EF
:1004C00000FF0000080808FF0000007028252970C0
:1004D0000070292529700070292528703E415D553E
:1004E000413E0AFB00FF000000FF00FF00000AFA87
:1004F00002FE00000A0B080F00000018246624000A
:1005000000292A7C2A29080808F800000000000FAA
:1005100008080808080F0808080808F80808000074
:1005200000FF0808080808080808080808FF080865
:1005300000205655567900702A252A71000F080BA5
:100540000A0A00FE02FA0A0A0A0B080B0A0A0AFA49
:1005500002FA0A0A00FF00FB0A0A0A0A0A0A0A0A41
:100560000AFB00FB0A0A005D2222225D0022555987
:10057000300000087F49413E007C55555544007CC1
:1005800055545544007C5555544400000007000064
:100590000000447D45000000457D45000000457C8D
:1005A00045000808080F0000000000F80808FFFFD9
:1005B000FFFFFFFFF0F0F0F0F0F000000077000028
:1005C0000000457D44000F0F0F0F0F0F003C42430A
:1005D0003D0000FE4A4A3400003C43433D00003DDC
:1005E00043423C000032494A3100003A4546390056
:1005F00000FC20201C0000FEAA28100000FFA524FB
:100600001800003C40413D00003C41413D00003DA0
:1006100041403C00009CA0613D00000408710904B9
:1006200000000202020000000703000000000808AA
:1006300008000000242E240000242424242405176C
:100640000A342A780006097F017F00224D5559227D
:100650000008082A08080000081818000006090900
:10066000060000000800080000000800000000026A
:100670000F00000000090F05000000090D0A00002E
:10068000003C3C3C3C0000000000000011241FBE68
:10069000CFEFD0E4DEBFCDBF11E0A0E0B1E0EAE4EF
:1006A000F2E100E00BBF02C007900D92A635B10742
:1006B000D9F725E0A6E5B1E001C01D92AC3BB20739
:1006C000E1F70E94C1050C9423090C940000FC0181
:1006D0001082758364837383628341834783468377
:1006E0000895FC0180818823B9F0A281B3819D0126
:1006F0002F5F3F4F8C919681915019F49181291B66
:1007000031093383228396832FB7F89490819150D7
:1007100090832FBF90E008958FEF9FEF0895FC0125
:10072000908181819817B8F4A481B5819D012F5FD4
:100730003F4F6C938781815019F48181281B3109C7
:100740008783358324839FB7F89480818F5F80836C
:100750009FBF81E0089580E0089587B18C7F87B9BD
:1007600088B1836088B983E08093B80087E0809384
:10077000B10082E0809370008DE78093B30078949D
:1007800008958AE08093560184EA8093BC0004C0F7
:100790008091BC0087FD04C0809156018111F8CF83
:1007A00080915601882329F08091B900887F90E0DC
:1007B00008958FEF9FEF08959AE0909356018093EC
:1007C000BB0084E88093BC0004C08091BC0087FD1E
:1007D00004C0809156018111F8CF80915601882381
:1007E00029F08091B900887F90E008958FEF9FEF06
:1007F00008950C94DC038AE08093560184E9809389
:10080000BC0008951F920F920FB60F9211248F9380
:100810008091B30083588093B30080915601882360
:1008200029F0809156018150809356018F910F904D
:100830000FBE0F901F9018958FB7F89427E630E001
:100840003093C5002093C40098E99093C10090ECC8
:100850009093C0008FBF40E16CEA71E084EA91E0C0
:100860000E94670340E464E671E08CE591E00C943B
:1008700067031F920F920FB60F9211240BB60F92BF
:100880002F933F934F935F936F937F938F939F9398
:10089000AF93BF93EF93FF936091C60084EA91E01A
:1008A0000E948F03FF91EF91BF91AF919F918F9124
:1008B0007F916F915F914F913F912F910F900BBE60
:1008C0000F900FBE0F901F9018951F920F920FB6AA
:1008D0000F9211240BB60F922F933F934F935F9378
:1008E0006F937F938F939F93AF93BF93EF93FF93F8
:1008F00080915C01811118C08091C1008F7D80932F
:10090000C100FF91EF91BF91AF919F918F917F9126
:100910006F915F914F913F912F910F900BBE0F9070
:100920000FBE0F901F9018958CE591E00E94710307
:100930008093C600E6CF8091570180FD0DC084B141
:10094000806A84B980E58CBD81E08DBD81E090E056
:10095000909358018093570108958EBD0DB407FE02
:10096000FDCF0895249A2C9A0C949B04BF92CF92A9
:10097000DF92EF92FF920F931F93CF93DF93BFB657
:10098000F8948CE3C82E85E0D82E97E0E92EF12C60
:100990000AC081E0E81AF10880E8C81AD1088FEF90
:1009A000E816F80621F180915B0190E00E2C02C060
:1009B000959587950A94E2F780FFEBCF4698479884
:1009C0008E2D806B0E94AD0480E10E94AD0480E01A
:1009D0000E94AD04479A860100581F4FE601899195
:1009E0000E94AD04C017D107D1F7469AD2CF10921A
:1009F0005B01BFBEDF91CF911F910F91FF90EF90F0
:100A0000DF90CF90BF900895ECEBF1E0CF018058DC
:100A10009F4F1192E817F907E1F785E0EC3BF807E3
:100A2000A9F78FEF80935B010C94B6048A3091F1A3
:100A30008D3069F13091590120915A0196E0899FDA
:100A4000F0011124E457FF4F86E0289FD0011124C4
:100A500090E8399FA00DB11D1124A454BE4F86E02B
:100A600094919D93815031968111FACF81E090E06D
:100A700001C0880F3A95EAF790915B01892B80932A
:100A80005B01243170F42F5F20935A010895109276
:100A90005A01089580915901873018F48F5F80932F
:100AA00059010895CF93DF93EC019881992339F090
:100AB0002196892F0E94160589918111FBCFDF9124
:100AC000CF91089580935A016093590108950E942F
:100AD000C10384EC0E94F90381E10E94DC0380E001
:100AE0000E94DC0380E00E94DC0380E00E94DC03C3
:100AF00080E00E94DC0380E00E94DC030C94FB0396
:100B0000CF930E949B0487B1806C87B9CFB7F894CC
:100B10004798469882EE0E94AD0483EA0E94AD0495
:100B200081E80E94AD0488E00E94AD0480EA0E9442
:100B3000AD0488EC0E94AD0485E20E94AD048FE212
:100B40000E94AD048FEA0E94AD04469A479A0E9423
:100B50000405CFBF0E94AD030E946705CF910C949E
:100B6000B204CF93C82F0E94C10384EC0E94F90302
:100B700085E10E94DC038C2F0E94DC03CF910C9452
:100B8000FB03CF93DF93CDB7DEB764970FB6F8942E
:100B9000DEBF0FBECDBF81B1877081B982B1886FD2
:100BA00082B98FE084B985B18F6085B90E941C0439
:100BB0000E948005789484E00E94B10581E0C12CF8
:100BC000D12C76019E012F5F3F4F490190E0A92E65
:100BD00091E0B92E0FC010E0813021F19FEFC91ACA
:100BE000D90AE90AF90A8FE99FE00197F1F700C0F5
:100BF0000000812F11E00399EECF882331F02FEF11
:100C0000C21AD20AE20AF20AEECF3FEF89EF90E071
:100C1000315080409040E1F700C00000C12CD12C41
:100C20007601EDCF2FEF39EF80E02150304080404A
:100C3000E1F700C000000E94040560E080E00E942F
:100C40006205FF92EF92DF92CF92BF92AF929F9296
:100C50008F920E943A06C4010E9452050E94B60477
:100C60000FB6F894DEBF0FBECDBFC12CD12C7601DC
:100C7000C394B9CF0F931F93CF93DF93CDB7DEB754
:100C80002E970FB6F894DEBF0FBECDBF0D891E891B
:100C900086E08C831A8309838FEF9FE79E838D8381
:100CA000AE01475E5F4F6F89788DCE0101960E943D
:100CB0006906EF81F885E00FF11F10822E960FB6BE
:100CC000F894DEBF0FBECDBFDF91CF911F910F9182
:100CD00008952F923F924F925F926F927F928F92E0
:100CE0009F92AF92BF92CF92DF92EF92FF920F93BB
:100CF0001F93CF93DF93CDB7DEB72B970FB6F89442
:100D0000DEBF0FBECDBF6C017B018A01FC011782E3
:100D10001682838181FFCCC1CE0101963C01F60190
:100D20009381F70193FD859193FF81917F01882342
:100D300009F4BAC1853239F493FD859193FF81910D
:100D40007F01853229F4B60190E00E948908E7CF3F
:100D5000912C212C312CFFE1F315D8F08B3279F056
:100D600038F4803279F08332A1F4232D20611DC044
:100D70008D3261F0803369F4232D216016C0832DFC
:100D80008260382EE32DE4603E2E2AC0F32DF860F9
:100D90001DC037FC2DC020ED280F2A3040F08E32C8
:100DA000B9F436FC81C1232D2064322E19C036FEE1
:100DB00006C08AE0989E200D1124922E11C0EAE010
:100DC0002E9E200D1124222EF32DF0623F2E08C0FE
:100DD0008C3621F4832D8068382E02C0883641F489
:100DE000F70193FD859193FF81917F018111B3CF2D
:100DF000982F9F7D9554933028F40C5F1F4F9FE3ED
:100E000099830DC0833631F0833771F0833509F053
:100E100059C021C0F801808189830E5F1F4F88244B
:100E20008394912C530113C02801F2E04F0E511C02
:100E3000F801A080B18036FE03C0692D70E002C0C9
:100E40006FEF7FEFC5010E947E084C018201F32DF8
:100E5000FF773F2E16C0280122E0420E511CF801F8
:100E6000A080B18036FE03C0692D70E002C06FEF34
:100E70007FEFC5010E9473084C01F32DF0683F2EEF
:100E8000820133FC1BC0822D90E088169906B0F4D5
:100E9000B60180E290E00E9489082A94F4CFF5011F
:100EA00037FC859137FE81915F01B60190E00E9489
:100EB000890821102A9421E0821A91088114910452
:100EC00071F7E8C0843611F0893641F5F80137FE34
:100ED00007C060817181828193810C5F1F4F08C0C0
:100EE00060817181072E000C880B990B0E5F1F4FDC
:100EF000F32DFF763F2E97FF09C090958095709552
:100F000061957F4F8F4F9F4FF0683F2E2AE030E072
:100F1000A3010E94C508882E861845C0853731F484
:100F2000232D2F7EB22E2AE030E025C0932D997F0D
:100F3000B92E8F36C1F018F4883579F0B5C08037F6
:100F400019F0883721F0B0C0E92FE061BE2EB4FE61
:100F50000DC0FB2DF460BF2E09C034FE0AC0292F3E
:100F60002660B22E06C028E030E005C020E130E067
:100F700002C020E132E0F801B7FE07C06081718154
:100F8000828193810C5F1F4F06C06081718180E078
:100F900090E00E5F1F4FA3010E94C508882E86189F
:100FA000FB2DFF773F2E36FE0DC0232D2E7FA22E68
:100FB000891458F434FE0BC032FC09C0832D8E7E98
:100FC000A82E05C0B82CA32C03C0B82C01C0B92C86
:100FD000A4FE0FC0FE01E80DF11D8081803321F4D5
:100FE0009A2D997EA92E09C0A2FE06C0B394B3948F
:100FF00004C08A2D867809F0B394A3FC11C0A0FE2A
:1010000006C0B21488F4280C922C9B180EC0B2149F
:1010100060F4B60180E290E00E948908B394F7CFB3
:10102000B21418F42B1802C0982C212CA4FE10C066
:10103000B60180E390E00E948908A2FE17C0A1FCDF
:1010400003C088E790E002C088E590E0B6010CC0DC
:101050008A2D867859F0A1FE02C08BE201C080E2A1
:10106000A7FC8DE2B60190E00E948908891438F44B
:10107000B60180E390E00E9489089A94F7CF8A94A1
:10108000F301E80DF11D8081B60190E00E9489080E
:101090008110F5CF222009F442CEB60180E290E023
:1010A0000E9489082A94F6CFF6018681978102C0B2
:1010B0008FEF9FEF2B960FB6F894DEBF0FBECDBF1C
:1010C000DF91CF911F910F91FF90EF90DF90CF9024
:1010D000BF90AF909F908F907F906F905F904F9058
:1010E0003F902F900895FC010590615070400110D1
:1010F000D8F7809590958E0F9F1F0895FC01615041
:10110000704001900110D8F7809590958E0F9F1F29
:1011100008950F931F93CF93DF93FB01238121FD4C
:1011200003C08FEF9FEF2CC022FF16C0468157816E
:10113000248135814217530744F4A081B1819D0178
:101140002F5F3F4F318320838C93268137812F5F20
:101150003F4F3783268314C08B01EC01FB010084D1
:10116000F185E02D0995892BE1F6D80116968D9130
:101170009C911797019617969C938E931697CE0184
:10118000DF91CF911F910F910895FA01AA2728307E
:1011900051F1203181F1E8946F936E7F6E5F7F4F44
:1011A0008F4F9F4FAF4FB1E03ED0B4E03CD0670FC0
:1011B000781F891F9A1FA11D680F791F8A1F911D13
:1011C000A11D6A0F711D811D911DA11D20D009F463
:1011D00068943F912AE0269F11243019305D3193A5
:1011E000DEF6CF010895462F4770405D4193B3E08E
:1011F0000FD0C9F7F6CF462F4F70405D4A3318F035
:10120000495D31FD4052419302D0A9F7EACFB4E0E5
:10121000A6959795879577956795BA95C9F700979D
:101220006105710508959B01AC010A2E069457953E
:10123000479537952795BA95C9F7620F731F841F95
:0A124000951FA01D0895F894FFCF3C
:10124A0074696D653A202564004A6F79737469631D
:10125A006B2055702E0D0A004A6F79737469636B9F
:10126A0020446F776E2E0D0A004A6F797374696392
:10127A006B204C6566742E0D0A004A6F7973746987
:10128A00636B2052696768742E0D0A004578697489
:06129A002E0D0A0A0000FF
:00000001FF
